:0600000000008A011E2829
:08000800090053347434613423
:100010007434693463342034643461347434613446
:100020003A34003420340034203443346F346D3497
:1000300070346C3465347434653400348330831622
:1000400081008B123930831290006030F800F2206A
:1000500029280D30FC200A30FC200530F00000304B
:10006000F10008210030F0000030F100831203138A
:100070007008A0002008F000F1011321831203137F
:100080007008A1007108A2002108F0002208F10008
:1000900020210930F0000030F100700823217108A0
:1000A0002321831203132008F000F1010130F20034
:1000B0000030F3002C213321F3003321F2003A21E8
:1000C0000319362803186928362883120313700889
:1000D000A0001230F0000030F10008210D30FC20AB
:1000E0000A30FC200030F0000030F10083120313CE
:1000F0007008A0002008F000F1017008F0007108FD
:10010000F10070082321710823212008F000F1017B
:100110003030F2000030F3002C2141211430F00087
:100120000030F1007008232171082321831203138A
:100130002008F000F1010130F2000030F3002C2122
:100140003321F3003321F2003A21031976280318F2
:10015000AE287628831203137008A0000030F00048
:100160000030F1007008A0002008F000F101132118
:10017000831203137008A1007108A2002108F00087
:100180002208F10020211430F0000030F100700846
:10019000232171082321831203132008F000F101A9
:1001A0000130F2000030F3002C213321F300332121
:1001B000F2003A210319B2280318E328B228831267
:1001C00003137008A0001430F0000030F100082183
:1001D0000D30FC200A30FC20E830F0000330F10044
:1001E0005E2172286730831603139900181598163C
:1001F0008312181698170800831203130C1EFE288A
:1002000099000800700FF103F10AF0007104080072
:100210000F21003803190800FC2002210829710869
:100220008A00700882008312031770088D008316FD
:100230008C010C140C181A2983120C08F000080009
:100240007008FC2008008B13F900780884007908F6
:100250008000F80A8B1708007208F007730803186B
:10026000730AF10708008B13F8037808840000086C
:100270008B17080073087102031D080072087002D2
:100280000800831603178C18432983123321332166
:100290008D0070088C0083168C130C1555308D0062
:1002A000AA308D008C148C1853290C110800F0030F
:1002B000700FF10AF1037008710408000B110B1D97
:0A02C0005F295721031D5E29080085
:10420000410042004300440045004600470048008A
:0442100049004A0017
:00000001FF
